:020000040800F2
:10000000C8060020C101000879080008750800082A
:100010007708000809050008F51000080000000036
:100020000000000000000000000000000D0B0008B0
:10003000C906000800000000E1080008810B000864
:10004000DB010008DB010008DB010008DB01000820
:10005000DB010008DB010008CD060008DB01000819
:10006000DB010008DB010008DB010008DB01000800
:10007000DB010008DB010008DB010008DB010008F0
:10008000DB010008DB010008DB01000800000000C4
:10009000000000000000000000000000DB0100087C
:1000A000DB010008DB010008DB010008DB010008C0
:1000B000DB010008DB010008DB010008DB010008B0
:1000C000DB010008DB010008DB010008DB010008A0
:1000D000DB010008410F0008DB010008DB0100081C
:1000E000DB010008DB010008DB0100080000000064
:1000F0000000000000000000000000000000000000
:1001000000000000000000000000000000000000EF
:100110000000000000000000DB010008DB01000817
:1001200000F002F800F03CF80AA090E8000C8244CD
:100130008344AAF10107DA4501D100F031F8AFF2AA
:10014000090EBAE80F0013F0010F18BFFB1A43F0B5
:10015000010318470425000024250000103A24BF9D
:1001600078C878C1FAD8520724BF30C830C144BF1C
:1001700004680C607047000000230024002500265E
:10018000103A28BF78C1FBD8520728BF30C148BFFA
:100190000B6070471FB502F0E3F91FBD10B510BD2D
:1001A00000F0B4F81146FFF7F5FF01F079FD00F01B
:1001B000D2F803B4FFF7F2FF03BC01F06EFD0000BC
:1001C0000948804709480047FEE7FEE7FEE7FEE7EB
:1001D000FEE7FEE7FEE7FEE7FEE7FEE70448054927
:1001E000054A064B70470000990B000821010008E2
:1001F000C8000020C8060020C8020020C802002055
:100200007047002000F03AF8FFF7C8FF012001F026
:1002100044FD10B5203AC0F00B80B1E81850203AE8
:10022000A0E81850B1E81850A0E81850BFF4F5AF96
:100230005FEA027C24BFB1E81850A0E8185044BF20
:1002400018C918C0BDE810405FEA827C24BF51F88D
:10025000043B40F8043B08BF7047D20728BF31F881
:10026000023B48BF11F8012B28BF20F8023B48BFD2
:1002700000F8012B704770477047704710B500F0C9
:1002800011F8BDE8104000F007B810B500F022F8F2
:10029000BDE81040AFF30080002801D001F0FDBCA4
:1002A0007047000010B5002102A000F05AF80120AC
:1002B00010BD0000534947414252543A2041626EFA
:1002C0006F726D616C207465726D696E6174696FB7
:1002D0006E00000010B5002102A000F042F80120DD
:1002E00010BD00005349475056464E3A2050757293
:1002F00065207669727475616C20666E2063616C2E
:100300006C65640000487047680000207546FFF780
:10031000F9FFAE4605006946534620F007008546C2
:1003200018B020B5FFF75AFFBDE820404FF0000697
:100330004FF000074FF000084FF0000B21F00701CD
:10034000AC46ACE8C009ACE8C009ACE8C009ACE810
:10035000C0098D4670470446AFF300802046FFF782
:1003600028FF70B505460C460A2000E06D1C01F020
:1003700095FC35B128780028F8D102E0641C01F022
:100380008DFC14B120780028F8D1BDE870400A2017
:1003900001F084BC004870476C000020002981688F
:1003A00002D041F0010101E021F0010181607047BC
:1003B0000D4910B5884202D1012144150AE00B49CC
:1003C000884202D10121041504E0094988420AD17A
:1003D0000121CC03204600F0BFFA2046BDE81040C2
:1003E000002100F0B9BA10BD0024014000280140EE
:1003F000003C01400029816802D041F4801101E0F5
:1004000021F4801181607047014600208968490706
:1004100000D501207047C06C80B2704702460020B2
:1004200012680A4200D00120704701460020896806
:10043000090700D50120704710B542680E4B1A40DD
:10044000D1E9003442EA04221343436082680B4B33
:100450001A40D1E9034323438C6842EA4402134320
:100460008360C26A097D22F47002491EC9B242EA61
:100470000151C16210BD0000FFFEF0FFFDF7F1FF6A
:1004800070B5072609290AD9C568A1F10A0404EB49
:100490004404A640B543A3401D43C56007E0056979
:1004A00001EB4104A640B543A3401D4305611F2352
:1004B000072A09D2446B521E02EB820293409C43EE
:1004C00091400C43446370BD0D2A09D2046BD21FC6
:1004D00002EB820293409C4391400C43046370BD45
:1004E000C46A0D3A02EB820293409C4391400C4354
:1004F000C46270BD816841F0080181607047816805
:1005000041F0040181607047FEE70000044B0122C6
:100510008240186809B1104300E0904318607047AA
:100520000074004010B501214C07204600F0FCF992
:100530002046BDE81040002100F0F6B930B5084C67
:10054000236840F6FE7282409343D1E900252A4396
:10055000D1E902510D432A4382401A43226030BD43
:1005600000740040014A10448160704700740040EC
:10057000014A10444161704700740040044A002958
:10058000516801D0014300E0814351607047000091
:10059000002004E00029016802D041F0010101E0DF
:1005A00021F0010101607047016821F00101016043
:1005B0000021016041608160C1603149304A0839E1
:1005C000904203D1486840F00F0006E02C4A1432F4
:1005D000904204D1486840F0F00048607047284AD3
:1005E0002832904203D1486840F47060F5E7244A0D
:1005F0003C32904203D1486840F47040EDE7204A15
:100600005032904203D1486840F47020E5E71C4A1C
:100610006432904203D1486840F47000DDE7184A24
:100620007832904203D1486840F07060D5E7154AAF
:10063000111F904203D1086840F00F0006E0114AF4
:100640001432904204D1086840F0F000086070470E
:100650000C4A2832904203D1086840F47060F5E7F4
:10066000084A3C32904203D1086840F47040EDE7FC
:10067000044A50329042EAD1086840F47020E5E71D
:100680000800024008040240406880B2704730B55C
:10069000036847F6F07293430C6A8A682243D1E9F3
:1006A00004452C4322438C692243CC6922434C6A83
:1006B00022438C6A22431A430260CA6842600A6875
:1006C00082604968C16030BD704700000249012066
:1006D000087000F003B800004400002001490860E1
:1006E000704700001404014030B51A4AC36801681D
:1006F00053B313688B431360111D0B680468A34345
:100700000B60416811440B68046823430B60114B74
:10071000083319680468A14319601C1D2168056825
:10072000A94321608168102905D011440A68006836
:1007300002430A6030BD19680268114319602168DC
:1007400000680143216030BD4068104402688A435C
:10075000026030BD0004014010B58A0721F0030497
:100760000649120F21440F238C6893409C438C60F0
:100770008B68904003438B6010BD00000000014077
:10078000F0B58C68002204F00F03E40601D54C6834
:1007900023430C884FF00F0C14F0FF0F4FF0010EA5
:1007A0001AD005680E880EFA02F42640A6420FD130
:1007B00096000CFA06F7BD4303FA06F635438E6839
:1007C000282E02D0482E02D002E0446100E00461ED
:1007D000521C082AE6D305600A88FF2A1DD94568FD
:1007E000002202F108060EFA06F40E882640A64200
:1007F0000FD196000CFA06F725EA070703FA06F56B
:100800008E683D43282E00D144618E68482E00D169
:100810000461521C082AE4D34560F0BDF0B5144CC5
:10082000002801DAE36900E06368420D120185B235
:10083000C0F301579540C0F30346032F05D0C20211
:100840000AD50322B240934307E023F07062636845
:1008500023F07063636002E0AB4343F0706201B168
:100860002A43002801DAE261F0BD6260F0BD0000B9
:1008700000000140FEE7FEE7FEE7000070B50F2430
:100880000178426801254FF0E026DAB1124A126879
:1008900002F4E062C2F5E062120AC2F10403D4403D
:1008A00042789A408378234013431A010B4BCA5471
:1008B000007800F01F018D40400906EB8000C0F871
:1008C000005170BD01F01F008540480906EB800013
:1008D000C0F8805170BD00000CED00E000E400E0C5
:1008E00070470000034A516821F4404101435160C0
:1008F0007047000000100240044A0029516901D0ED
:10090000014300E081435161704700000010024044
:10091000044A0029D16901D0014300E08143D1613B
:100920007047000000100240044A0029116901D0FC
:10093000014300E081431161704700000010024054
:10094000044A0029916901D0014300E0814391618B
:100950007047000000100240044A0029D16801D00D
:10096000014300E08143D160704700000010024065
:1009700030B5224A5168224B11F00C0103D00429F2
:1009800001D0082901D0036015E05168546801F4D2
:1009900070114FF0020514F4803F05EB914107D030
:1009A000D46A04F00F04641CB3FBF4F34B43EAE78E
:1009B000144B594301605168134B01F0F0010909D0
:1009C0005C5C0168E1404160546804F4E064240A1E
:1009D0001C5D21FA04F48460546804F46054E40A51
:1009E0001B5DD940C1605268074B02F44042920B34
:1009F0001B1F9A5CB1FBF2F1016130BD0010024097
:100A000000127A0000093D004A0000203EB504466D
:100A10000B48012150F82400FFF792FF084869466F
:100A20000A3830F81400ADF80000102002900320BE
:100A30000190044850F82400FFF7A2FE3EBD0000DC
:100A400084250008080000200349044A31F81010EA
:100A500052F82000416170477A2500080800002004
:100A60000349044A31F8101052F820000161704720
:100A70007A2500080800002030B5044621480D46BC
:100A800089B050F82400012140F00100FFF758FF21
:100A9000042008901B4806A90C3830F81400ADF863
:100AA0001800194850F82400FFF76AFE012D27D1DD
:100AB0001448103830F81400C1B212480E3830F81B
:100AC0001400C0B2FFF748FE0E480A3830F8140090
:100AD0000090002001900820CDE902056846FFF74C
:100AE00003FE0848083830F814008DF810000F2075
:100AF0008DF811008DF8120004A80595FFF7BEFED1
:100B000009B030BD802500080400002070470000B7
:100B10001A4900200A6842F480320A604FF4A06348
:100B20000A6800F1010012F4003F01D19842F7D1A8
:100B30000868800321D5486848604868486048686C
:100B40004860486820F47C104860486840F4981079
:100B50004860086840F08070086008688001FCD533
:100B6000486820F003004860486840F00200486090
:100B70004868C0F381000228FAD170470010024093
:100B80000448407800284FF0000001D0FFF768BF0C
:100B9000FFF75ABF44000020104810B5016841F02B
:100BA0000101016041680E4A1140416001680D4A2F
:100BB00011400160016821F480210160416821F445
:100BC000FE0141604FF41F0181600021C162FFF707
:100BD0009FFF05494FF00060086010BD0010024003
:100BE0000000FFF8FFFFF6FE08ED00E00029018895
:100BF00002D041F0800101E021F0800101807047C6
:100C00000029018802D041F0010101E021F0010139
:100C100001807047002930F8441F02D041F40041A0
:100C200001E0C1F30E010180704700004B4910B58F
:100C3000884202D10121C41486E0B0F1804F09D06E
:100C4000474988420DD101210220FFF76DFE0021A6
:100C5000022064E001210846FFF766FE0021012022
:100C60005DE04049884206D101210420FFF75CFE87
:100C70000021042053E03C49884206D1012108208C
:100C8000FFF752FE0021082049E03849884206D18A
:100C900001211020FFF748FE002110203FE03449D9
:100CA000884206D101212020FFF73EFE00212020AE
:100CB00035E03049884202D10121441444E02E49F4
:100CC000884202D10121CC043EE02C49884202D165
:100CD00001210C0538E02A49884202D101214C0546
:100CE00032E02849884206D101214020FFF71CFE4E
:100CF0000021402013E02449884206D101218020B0
:100D0000FFF712FE0021802009E0204988420AD125
:100D1000841501212046FFF707FE00212046BDE88B
:100D20001040FFF701BE1A49884202D101210C048C
:100D30000AE01849884202D101214C0404E0164916
:100D400088420AD101218C042046FFF705FE204687
:100D5000BDE810400021FFF7FFBD10BD002C014091
:100D60000004004000080040000C0040001000405B
:100D70000014004000340140004C0140005001408C
:100D80000054014000180040001C004000200040BA
:100D900000400140004401400048014030B5028C51
:100DA00022F010020284028C8388048B22F020023D
:100DB00024F4E6450C88240645EA14440D892D05E3
:100DC00042EA15454A88120545EA1242104DA842EA
:100DD00002D0104DA84215D122F080054A8923F493
:100DE0004063120545EA124222F040058A88120546
:100DF00045EA12428D89AD0443EA1545CB899B042F
:100E000045EA134383800483C9880187028430BD87
:100E1000002C01400034014030B5028C22F4805295
:100E20000284048C8288838B23F4E6450B881B069E
:100E300045EA134324F400550C89240745EA144479
:100E40004D882D0744EA1545094CA04202D0094CB3
:100E5000A04205D122F480448A89920544EA1242D4
:100E600082808383C988A0F84010058430BD0000CB
:100E7000002C014000340140828B22F4006242EADF
:100E800001218183704781857047A0F84010704729
:100E900030B502881B4C1C4DA0420DD0A8420BD08F
:100EA000B0F1804F08D0194B984205D0184B9842AA
:100EB00002D0184B984203D122F070034A881A439B
:100EC000154B984206D0154B984203D022F440733C
:100ED000CA881A4302808A8882850A880285A042CD
:100EE0000AD0A84208D00E4A904205D00D4A90423E
:100EF00002D00D4A904201D1097A018601218182F6
:100F000030BD0000002C01400034014000040040CE
:100F100000080040000C0040001000400014004099
:100F20000040014000440140004801404FF6FF717D
:100F3000818000210180C1804180017270470000E2
:100F40000E4810B50188890616D5018821F02001C8
:100F50000180011D09880A4CCAB26168094B0B4423
:100F6000491C61601A70712A06D10021616032212A
:100F700000F0B5F80120207010BD000000380140DD
:100F8000100000205C00002010B5028A4FF2FF0321
:100F90001A400B884C8823438C88C9880C43234310
:100FA0001343038210BD0021018041808180C180F4
:100FB00070470029818902D041F4005101E021F4F9
:100FC000005181817047002A828A01D00A4300E0E3
:100FD0008A43828270470246002012880A4200D06B
:100FE0000120704710B5C1F3421301F01F04012125
:100FF000A140012B07D0022B07D01430002A026831
:1010000005D00A4304E00C30F8E71030F6E78A43D5
:10101000026010BD30B50D46018A85B004464CF61D
:10102000FF700140E88808432082A0894EF6F31142
:101030000840A9882A8911436A8902431143A18182
:10104000A18A4FF6FF400140A8890843A082684664
:10105000FFF78EFC1B48844201D1039800E0029800
:10106000A1890904002900EBC00101EB00102968E7
:1010700002DA4FEA410101E04FEA8101B0FBF1F0F1
:101080006422B0FBF2F14FEA01114FEA11136FF045
:1010900018056B4300EB8300A3891D044FF0320356
:1010A00006D503EBC000B0FBF2F000F0070005E04E
:1010B00003EB0010B0FBF2F000F00F0008432081BA
:1010C00005B030BD003801404FF4165101600021D9
:1010D0008180C18001810C2242818181704700B5ED
:1010E0000346C8B2988080211846FFF774FF002895
:1010F000F9D000BDFEE72DE9F0410446884600F036
:101100007BFD06464146204600F04CF80546414628
:10111000204600F02DF807464146204600F00CF826
:1011200004F5967406EB050021683844C4E90051C3
:1011300080F30C00BDE8F08110B5012200EB420302
:10114000521CB3F83241A3F83441062AF6D3A0F872
:10115000341110BD0022C0F830211146C0F82C21F6
:1011600000EB4103491CA3F834210629F8D370474A
:1011700030B5B0F93641CD1701EB157104EB2111F3
:10118000B0F93A41B0F93E21091BD41702EB1472B1
:10119000D0F8243101EB2211D0F828014B4393FB06
:1011A000F0F030BD2DE9F34F00F58E7481B060682A
:1011B00000F0D7FF81468846606900F0D2FF0646FE
:1011C0000F46B4F91A0000F0CCFF1A4A1A4B00F08F
:1011D000DFFF05460091B4F9180000F0C2FF174A7E
:1011E000174B00F0D5FF82468B46029800F0B9FFFE
:1011F000104A114B00F0CCFF52465B4600F082FDD6
:101200002A46009B00F07EFD32463B4600F07AFD08
:1012100005460E46206800F0A4FF2A46334600F03B
:10122000B7FF4A46434600F015FE03B0BDE8F04F55
:1012300000F068BFC7BAB88D06F0D63F9CA223B9AC
:10124000FC87F43F38B5049C009400F0FDF8034996
:10125000016040F2DC51A0F8101138BDD025000823
:10126000FEB50E461546044600F0D2FC07B2EDB1BD
:10127000D4E945010144714391FBF0F0C01B01B278
:101280002068C26920469047051E00DA002081B21E
:10129000204600F0B9FC2B4632463946684600F03D
:1012A000AFFA6946201D00F0D9FBFEBD3046E5E7E8
:1012B0002DE9F74F84B004466FF0270B9EE02068BD
:1012C0008169204688470121204600F013FA04F581
:1012D00082700021074600F0D7FA002104F58070E3
:1012E00000F0BCFC204600F097FC05460421204697
:1012F00000F000FA00260121384600F0C5FA4C2D16
:101300003AD004DC422D33D0492D04D138E0502DA1
:101310003AD0542D28D03DA1201D00F0B9FB4FF448
:101320007A704FF0280800254FF4006640F6FF77EA
:10133000C246D946C4F80C013B46324629466846A7
:1013400000F05EFA6946201D00F088FB05EB0800FE
:1013500005B206EB0A0006B207EB090007B2002D42
:101360002DDA4FF028082EE0204600F0C1F842E0C8
:10137000204600F037F93EE0204600F007F93AE059
:10138000204600F0DBF836E028A1201D00F080FBAD
:101390004FF47A70C4F80C01226831462046D268B6
:1013A000761C09B2904701462046069AFFF758FF7F
:1013B000D4F80C01401EC4F80C01EDD11BE0B5F5CA
:1013C000805F00DBD846002E02DA4FF0280A03E0E7
:1013D000B6F5805F00DBDA46002F02DA4FF028090D
:1013E00003E0B7F5805F00DBD946D4F80C01401E5E
:1013F000C4F80C01A0D1201D00F0FAFA05980028CD
:101400007FF45DAF07B0BDE8F08F000044657A65FA
:10141000206F70746965206973206E696574206936
:101420006E206765627275696B0000005049442D3B
:10143000526567656C616172206D657420737461BB
:1014400070696E7075740A002DE9FC4115461E46E0
:10145000089F00F0F3F80446104844F8AC0BD5E9B7
:101460000001C4E91A01D6E90001C4E91C01D7E969
:101470000001C4E91E01A4F1AC044FF001024FF0D9
:101480000001684600F0B1F90146284600F0C7FBAC
:1014900010B12046BDE8FC81FEF7B3FEF825000838
:1014A00000F5827000F0E5B9FEB50C46054600F087
:1014B000AFFB0646A1B2284600F0A6FB0023224659
:1014C0003146684600F09CF96946281D00F0C6FACE
:1014D000FEBD000010B500F02FF9034901604FF484
:1014E0007A71C0F80C1110BD20260008704700006A
:1014F00070B504460DA1001D00F0CAFA4FF47A70D1
:101500000025C4F80C01226829462046D2686D1CCB
:1015100009B2904701462046FFF7C6FFD4F80C01F8
:10152000401EC4F80C01EED170BD00005374617010
:10153000726573706F6E73696500000070B5044664
:101540000DA1001D00F0A4FA4FF47A700025C4F834
:101550000C0122682946204692686D1C09B290470A
:1015600001462046FFF7A0FFD4F80C01401EC4F846
:101570000C01EED170BD0000496D70756C73726521
:1015800073706F6E7369650A0000000070B50446E1
:101590000FA1001D00F07CFA012104F5827000F01B
:1015A00073F94FF47A700025C4F80C0122682946BB
:1015B000204612696D1C09B2904701462046FFF78C
:1015C00073FFD4F80C01401EC4F80C01EED170BDBD
:1015D00048656C6C696E67726573706F6E73696570
:1015E0000A00000070B504460FA1001D00F050FA7B
:1015F000012104F5827000F047F94FF47A7000255C
:10160000C4F80C0122682946204652696D1C09B2B3
:10161000904701462046FFF747FFD4F80C01401ED3
:10162000C4F80C01EED170BD426C6F6B676F6C66D5
:10163000726573706F6E73696500000010B5FFF717
:1016400049FF034901600021A0F8101110BD0000FE
:101650003026000830B58BB001210220FFF758F981
:101660004FF40070ADF81C0018200990022008907B
:1016700007A91D48FFF784F801211C48FFF7CEF8A1
:101680001B4D2846FFF7D2FA42F6E060ADF8140091
:101690004FF47A70ADF810000024ADF81640ADF8A4
:1016A000124004A92846FFF7F3FB6020ADF80000C4
:1016B0000120ADF8020041F27070ADF80600ADF8FF
:1016C000084069462846FFF7A7FB08212846FFF790
:1016D000D3FB01212846FFF789FA01212846FFF7AD
:1016E0008FFA0BB030BD000000100140000C1A0052
:1016F0000004004070B5052901DBFEF782FD0C48AF
:1017000089B10C4A054632F811400121FFF778FAF9
:101710006004010C2846FFF7B6FB21462846BDE8C9
:101720007040FFF7B2BBBDE870400021FFF768BA18
:1017300000040040BC25000810B50C46194902C041
:1017400000F0CCF900222146FC3000F01BF9052204
:101750002146001D00F09CF8A0F5827472B60020AE
:10176000FFF754F90020FFF76FF90120FFF74EF95A
:101770000120FFF769F901210020FFF77DF9012120
:101780000846FEF7FBFE01210220FEF7F7FE0121CD
:10179000C802FEF7F3FE2046FFF75CFF62B6204664
:1017A00010BD00005026000810B503E0521049108B
:1017B000C0E900210268D10702D14168CB07F5D00A
:1017C000032101E0C0E90023036893FBF1F201FB70
:1017D000123333B9446894FBF1F301FB1344002C3A
:1017E000F0D0891C0929EFDB10BD10B50446C4E90F
:1017F00000121AB1FFF7D8FF204610BDFEF701FD19
:1018000009BA016011BA416019BA8160704710B518
:1018100004464FF6FF7088B0814201D3FEF7F1FC19
:10182000A1806846FFF782FBA088ADF804000C2079
:10183000ADF800000020ADF80600ADF802006946E2
:101840002068FFF725FB6020ADF80C000120ADF803
:101850000E00A088ADF812000220ADF8140003A914
:101860002068FFF79BFA01212068FFF7D3F908B041
:1018700010BD4FF6FF72914201D3FEF7C2FC4FF448
:101880007A725143FFF7C3BF0068FFF7B9B9000090
:1018900070B505468AB04FF0804028600C46AA809B
:1018A00001214015FFF74CF80020FFF71BF83248E4
:1018B000002CD0E9031240690691CDE9072051D0F0
:1018C000012C51D0022C01D0042C4FD00421ADF8B2
:1018D000181006A92948FEF753FFECB3012C04D0D9
:1018E000022C02D0042C45D00224254E3046FEF7AF
:1018F0005FFD2149182218316846FEF78AFC6946C7
:101900003046FEF799FD0723012221463046FEF7B7
:10191000B7FD01213046FEF76DFD01210846FEF7B7
:10192000F7FFA9882846FFF7A4FF01213046FEF7FC
:1019300035FD00212868FFF763F93046FEF7DAFD30
:101940003046FEF772FD0028FAD13046FEF7D7FD8B
:101950003046FEF759FD00E00AE00028F8D10AB051
:10196000284670BD4021B2E70221B0E78021AEE7F2
:101970000624BAE70724B8E78C25000800080140D0
:101980000024014030B587B00C46016005460121B6
:101990004807FEF7BDFFFEF7C5FD1349D1E9000278
:1019A0008968CDE904020691C4B11020ADF8100099
:1019B00004A90E48FEF7E4FE002200920192029272
:1019C00003926CB100206946FEF7B8FD54B10020C7
:1019D0000121FEF79BFD07B0284630BD2020E5E73A
:1019E0001020F0E71020F3E78C25000800080140E4
:1019F00070B5184D04462846FEF746FE0028FAD179
:101A000000212846FEF7C6FD1349B4F8F800C86067
:101A100094F8FA00C0EB001004EBC00008304860F6
:101A20002846FEF734FE01212846FEF7B3FD94F860
:101A3000FA00012801D0012000E0002084F8FA001B
:101A4000C0EB001004EBC000083060600020A4F878
:101A5000F80070BD440002401800002070B5044634
:101A6000B0F8F8000D46782802D12046FFF7C0FFF5
:101A700060682968016069684160A9688160606880
:101A80000C306060B4F8F8000C30A4F8F80070BDB9
:101A900030B4002204E04468A354521C1D2A0AD228
:101AA0008B5C0BB10A2BF6D120211D2A03D243688F
:101AB0009954521CF9E742680A2151771E21A0F877
:101AC000F81030BCFFF794BF10B504460146024839
:101AD000FFF705FB204610BD003801402DE9F0411D
:101AE00004468CB00830606001270026A4F8F86036
:101AF00084F8FA7039463846FEF7FEFE012144F2BA
:101B00000400FEF71DFF182002904FF49050DFF8FC
:101B10009880ADF800000225694640460195FEF721
:101B20002FFE482002904FF44060ADF80000694657
:101B300040460195FEF724FE09A8FFF734FA1B4D35
:101B400009A92846FFF720FA03A8FFF7BDFA4FF4CA
:101B5000612003904FF44070ADF8180003A92846A7
:101B6000FFF758FA25208DF81C008DF81E60042020
:101B70008DF81D0007A80897FEF780FE012240F2AD
:101B800025512846FFF72EFA012280212846FFF72B
:101B90001AFA0748FEF708FD01212846FFF709FA5F
:101BA0000CB02046BDE8F08100080140003801403B
:101BB00044000240B0F8100100B2704709B10020A3
:101BC000704740F6D8607047880000B27047000048
:101BD000084AB2F90010402902DA40F6087000E025
:101BE000F820491C09B211807F2901DD00211180F4
:101BF0007047000000000020D0F81421D0F8180130
:101C00004A4392FBF0F0704700F5807000F026B870
:101C100000F5827000F012B8001D00F02DB8884267
:101C200009D00A6803689A4203D149684068814232
:101C300001D00120704700207047000010B5064C0D
:101C400002212046FEF7EAFB0028F9D02046BDE835
:101C50001040FEF7E0BB000000240140B1F5805FBA
:101C600001D340F6FF71006800284FF0000001D05A
:101C7000FEF778BCFEF77CBC044820BF0178002941
:101C8000FBD000210170024800787047100000204E
:101C90005C0000200020FEF7F8BAFEE700F02DB847
:101CA00030B5D7B00322022155A8FFF79EFD0446A8
:101CB0001022012153A8FFF798FD054601220521B6
:101CC00051A8FFF792FD02462B46002101A800947F
:101CD000FFF7B8FA4FF40060ADF81401052101A830
:101CE000FFF7DEFB0122114601A8FFF7E1FA01A888
:101CF000FFF7FCFB57B0002030BD0021C0B2FFF75A
:101D0000E3BE000010B591EA030F48BF83F0004323
:101D100000F14483841A71EB030C05D2121943EBD2
:101D20000C03001B61EB0C01DFF824E14FEA1154B6
:101D3000A4EB135C1EEA430F18BF9EEA445F73D006
:101D400023EA0E03DCF1200E21EA045143F4801350
:101D500032D322FA0CFE10EB0E0023FA0CFE41EBFC
:101D60000E01CCF1200E03FA0EFE10EB0E0051F125
:101D70000001B1F5801FCCF1200E32D201EB0451ED
:101D800012FA0EF2BDE8104058BF7047401C38BF31
:101D90005FEA420218BF7047002814BF20F001001C
:101DA00041F100014FEA410313F5001F38BF7047AE
:101DB000A1F1C04100F0E4BA012A43EB0302ACF107
:101DC000200CDCF11F0E32BF4FF0000E23FA0CF393
:101DD00010EB030041EB0451B4EB115FD0D0A1EB49
:101DE000045101F5801149085FEA300001EB04510C
:101DF0000ED350F1000038BF12FA0EFE08D1BDE834
:101E00001040C9E7401C38BF5FEA4202CAD1C3E7AD
:101E1000BDE810404FEA410313F5001F38BF70477B
:101E2000A1F1C04100F0ACBA9EEA445F08D011EACB
:101E30005E0FBDE8104004BF01F000410020704774
:101E4000BDE8104070B500F04DFA00BF64FBBE3E27
:101E50000000E0FF2DE9C04130B4DFF8A0C23CEA49
:101E6000111418BF3CEA131400F0EC8081EA03055A
:101E70001CEA111444EAD57418BF1CEA131500F0CB
:101E8000C780A4EB05044FF0004545EAC12145EAAF
:101E9000C32341EA505143EA525304F17F749942FB
:101EA00004F500344FEAC0204FEAC22208BF904236
:101EB00000F09C804FEA13650FF24016765D4FEA02
:101EC000134506FB05F7C7F1807706FB07F74FEAD6
:101ED000D737A7FB03687642C8F58038A7FB06CE44
:101EE00038BFA8F1010807FB08E64FF0000EA6FB7B
:101EF000028CE6FB03CEDCF1000CCEF1004E38BFC5
:101F0000AEF1010EA6FB0C584FF000074FF0000594
:101F1000E6FB0E87A1FB08C6A0FB07CE16EB0E065C
:101F200045F10005E1FB076515F1E04E7EBFA4F524
:101F300080345FEA46066D4116F1800745F10005E1
:101F40004FEA17274FEA066647EA0567A6F1DE461D
:101F5000B6F1805F4FEA15251FD9384624F0010CF1
:101F600005EBC471BCF1FE6F01EB0C1102D8F0BCA3
:101F7000BDE8008124425CBF01F5801E9EEAC47F5B
:101F800002D4F0BCBDE80081244238D4F0BCA1F1F9
:101F9000C041BDE8004100F0F3B94FEAD22242EA65
:101FA00043524FEAD323A7FB02864FEAD02040EAF0
:101FB000415007FB03661EEA0E0F4FEAD12105FBD5
:101FC000026658BFA6EB0056B6EB00564FEA520E1B
:101FD0004EEAC37E18EB0E0E56EB530EBDD518EB32
:101FE00002085E417F1C55F10005B6E74FF48015ED
:101FF0004FF000074FF000064FF00008ADE7F0BCCF
:102000004FF0000001F1C04101F00041BDE8008146
:1020100011EA0C1F0CEA131500D00CE013EA0C1F98
:1020200000F025804FF00000F0BC81EA030101F0D0
:102030000041BDE80081F0BCBDE8004181EA030138
:1020400000F09EB9F0BCBDE8004170B500F04AF95F
:10205000097EFC3E00F007B881EA03014FF0000062
:1020600001F00041704781EA030100F089B9F0BC3A
:10207000BDE800414FF0000021497047FFFDFBF92A
:10208000F7F5F4F2F0EEEDEBE9E8E6E4E3E1E0DEAB
:10209000DDDBDAD8D7D5D4D3D1D0CFCDCCCBCAC81D
:1020A000C7C6C5C4C2C1C0BFBEBDBCBBBAB9B8B744
:1020B000B6B5B4B3B2B1B0AFAEADACABAAA9A8A837
:1020C000A7A6A5A4A3A3A2A1A09F9F9E9D9C9C9B05
:1020D0009A999998979796959594939392919190B0
:1020E0008F8F8E8E8D8C8C8B8B8A89898888878741
:1020F0008685858484838382828181800000FF07B6
:102100000000F87F4FEA41034FEA5353A3F5806381
:10211000D3F11E03C8BFD3F1210C0CDD4FF00042F8
:1021200042EAC12242EA505232FA03FC8CEAE17CD4
:10213000ACEBE1707047102BC4BF0020704703F573
:10214000787CBCF1FF3F04D06FF0004282EA2100AE
:10215000704770B500F0C6F849922480002070479F
:10216000F2E710F0004248BF4042B0FA80F310FAA4
:1021700003F10AD0C3F11D0303F580634FEA415018
:1021800002EB035202EBD12170474FF00000704781
:10219000DFF848C170B51CEA111E1EBF1CEA1315FA
:1021A0009EEA0C0F95EA0C0F00F06F8081EA0304A1
:1021B00023EA4C134EEAD47E21EA4C1141F48011FB
:1021C00043F48013AE44A1FB024CA0FB0365AEF1C7
:1021D0007F7E361955EB0C05A1FB034C4CF1000337
:1021E000A0FB021C16EB0C06654153F100030942EB
:1021F00018BF46F0010613F4007F0BD14FEA0331FC
:102200004FEA0530340341EA155140EA16506FF0A9
:1022100003020AE04FEAC3214FEAC520F40241EA73
:10222000555140EA56506FF0020202EB2E4201EB8C
:10223000025585EACE710AD05FEA440C18BF24F03B
:10224000004450F1000041F1000120EAD47040F256
:10225000FE7C624500D270BDA84214BF4FF080449E
:102260004FF04044002E08BF0024BEF1806FA8BF8D
:10227000A1F1C041BDE8704080F282804FF00000C3
:1022800001F1C04101F0004170479EEA0C0F0CEAD9
:10229000131518BF95EA0C0F06D04FF0000081EA25
:1022A000030E0EF0004170BD00F01CF88900013EE5
:1022B00000F007B800F009B84FEA430C5FEA5C5C35
:1022C00008D081EA030100F05BB84FEA410C5FEAF5
:1022D0005C5CF6D14FF00000014970470000FF0739
:1022E0000000F87F0EF1020E2EF0030E5EF8046B74
:1022F000364205D4012A43EB030515F5001F12D819
:10230000012841EB010C1CF5001F0CD80ED14FEA3F
:10231000D17C15F5001F0CEB4C0C0CF1020C08BF26
:102320004CEBD37C04E04FF0080C01E04FEAD37C87
:102330000CEB4C0526FA05F606F00706B6F1040C80
:1023400006D20EEB860CBDE870404CF0010C6047E5
:10235000DFE80CF0090B02024FF000414FF00000E3
:10236000A1F5002170BD19461046012851EB01046A
:1023700018BFD4F5001484BF002001F0004170BDE7
:102380000808A0F500114FEA3101704710B591EA35
:10239000030F48BF83F000433FF5BCAC841A71EBD8
:1023A000030C07D212198CF0004C43EB0C03001BFA
:1023B00061EB0C01DFF8A4E14FEA1154A4EB135CCC
:1023C0001EEA430F18BF9EEA445F00F0B08023EA84
:1023D0006E03524221EA0451C3EB6E0338BF5B1E09
:1023E000DCF1200E25D322FA0CFE10EB0E0043FA8E
:1023F0000CFE41EB0E01CCF1200E03FA0EFE10EBA9
:102400000E0051F10001CCF1200E29D412FA0EF287
:1024100001EB0451BDE8104058BF7047401C1CBF81
:10242000B2F1004F704700280CBF491C20F001009A
:10243000704712EB020E43EB030218BF4FF0010E80
:102440004EEA4202ACF1200CDCF11E0E54D943FAE4
:102450000CFE10EB0E0051F1FF31CCF11E0ED5D564
:102460000EF1010E12FA0EFE404141EB010101EBAB
:10247000445C5FEA5C5C10D910EBDE7001EB045148
:1024800038BFBEF1004FBDE8104018BF70470028AC
:102490000CBF491C20F00100704730D24FEAD42C09
:1024A00011F5001124F400641BD0B1FA81F20B3A4B
:1024B000A41AA41ED2F12003914030FA03F3194369
:1024C000904001EBCC71002C01EB0451BDE81040B1
:1024D000A8BF704701F1C0414FF0000001F000417A
:1024E0007047B0FA80F310FA03F100D110BDE41A7E
:1024F000173C4805C90AE4E701EB045110BD491037
:1025000001EB0451BDE810404FEA300002E04FF00B
:10251000000170474A0008BF0042F8D0B2F5001F22
:1025200028BF704701F000414FF0000070479EEA5D
:10253000445F07D011EA5E0FBDE8104004BF0021E0
:1025400000207047BDE8104070B5FFF7CBFE00BF1C
:1025500040DFF63E83F00041104670470000E0FF88
:1025600010B5FDF717FF4FF00001016010BD00002E
:102570000000000001000100060000020001000050
:102580000400000010000000100000000000000027
:102590000200000010000000000000000300000026
:1025A000000000000000000000000000000000002B
:1025B0000000060000000000010000000000E02E06
:1025C0007017B80BE80300000000000000000000D6
:1025D0000000000000000000BD1B0008B51B000843
:1025E000C91B0008D11B000855110008F71000088E
:1025F00000000000000000000000000000000000DB
:10260000951C0008951C0008951C0008951C0008E6
:10261000951C0008951C0008000000000000000048
:10262000ED140008000000000000000000000000A1
:102630000000000000000000951C0008951C000828
:10264000951C0008951C0008000000000000000018
:1026500000000000000000007826000800000020B4
:102660005C0000005C010008D42600085C0000202B
:102670006C0600007801000800000000000801401E
:1026800000100140001001400000000000000000A8
:1026900004380140000000001000000000000000AD
:1026A00000000000800000000000000000000000AA
:1026B00000000000002000000000000000000204F4
:1026C00006080000000001020304010203040607DB
:0426D00008090000F5
:0400000508000121CD
:00000001FF
